:020000040800F2
:1000000000500020151500081315000811150008F0
:100010001115000811150008111500080000000056
:1000200000000000000000000000000013150008A0
:100030001315000800000000131500081315000830
:1000400011150008111500081115000811150008F8
:1000500011150008111500081115000811150008E8
:1000600011150008111500081115000811150008D8
:1000700011150008111500081115000811150008C8
:1000800011150008111500081115000811150008B8
:1000900011150008111500081115000811150008A8
:1000A0001115000811150008111500081115000898
:1000B0001115000811150008111500081115000888
:1000C0001115000811150008111500081115000878
:1000D0001115000811150008111500081115000868
:1000E0001115000811150008111500081115000858
:1000F0001115000811150008111500081115000848
:100100001115000811150008111500081115000837
:100110001115000811150008111500081115000827
:100120001115000811150008111500081115000817
:100130001115000811150008111500081115000807
:1001400011150008111500081115000811150008F7
:1001500021217F22014B00F0EBBB00BFD901000839
:100160002DE9F0411A4E3378042B03D0072B2DD004
:10017000BDE8F081174C00F0B7FAB4F808346BB959
:100180002378212B05D0412B1AD1D4F8010000F09F
:1001900031F9D4F80130C4F8043411E0A046D4F8A1
:1001A0000424023B02EB83270025B4F800349D426F
:1001B00006DAE81938F8051000F0ECF80235F4E733
:1001C00000F0A4FA05233370BDE8F08101F0EAF9EC
:1001D000000000202004002038B5087800F07F00DF
:1001E000212852D14878013805284ED8DFE800F0A0
:1001F000034D241A4620274D0BB1188808B9062351
:100200000EE08C78C978244844EA0121A0F808144B
:100210001988A0F8001411681A8801F0CBF903239B
:100220002B7034E01B4B1A780A2A30D1022201E0ED
:10023000184B02221A702AE016481568047800212B
:10024000032C04D0062C06D10724047003E00424F8
:100250000470642400E00C462970156800786C7006
:100260001468A1701468E1701468207112685171EB
:1002700006221A80094A049B1A6008E005491268A0
:10028000097801201170188038BD002038BD012088
:1002900038BD00BF000000202004002061010008DC
:1002A00030B540F2023085B000F007FA224B234A05
:1002B00019681C46914210D0214A224B11680B400C
:1002C000B3F1005F09D1204B4FF40051196013685E
:1002D00083F308881D4B1B6898470025256000F0B4
:1002E000A1F94FF4417000F0E8F92A464FF4006399
:1002F0001748032100F0BAF815484FF4006100F0E8
:10030000D3F904230093134B134901934FF48063F3
:100310000293124A124B134800F006FA124904469F
:1003200000F0A7FD0A484FF4006100F0BFF9204635
:1003300000F026FAFBE700BF004C0020ADDEE1FE36
:10034000002000080000FE2F08ED00E00420000857
:100350000010014020000020FC1600080E170008C5
:10036000040000200018000851010008064B18681E
:10037000064B1B68B3F5007F82BF054B1B68184313
:1003800000F03500704700BF0C200240E0F7FF1F6F
:100390004C20024038B504460D4600F0BFF9114B21
:1003A0001B68B3F5007F04D90F4B9C4201D90F4A5B
:1003B00000E00F4A136843F001031360258000F04A
:1003C000ADF9084B1B68B3F5007F04D9064B9C427E
:1003D00001D9064A00E0064A136823F001031360BE
:1003E00038BD00BFE0F7FF1FFFFF070850200240A5
:1003F0001020024010B5044600F090F9154B1B6820
:10040000B3F5007F09D9144B9C4206D9134B1A68E7
:1004100042F002021A60124A05E0124B1A6842F0DA
:1004200002021A60104A14601A6842F040021A6010
:1004300000F074F9074B1B68B3F5007F04D9064B35
:100440009C4201D9054A00E0064A136823F00203E2
:10045000136010BDE0F7FF1FFFFF070850200240A8
:100460005420024010200240142002402DE9F047A1
:100470004FF6E07796469C460268436800264FF0A8
:100480000F084CFA06F4E40719D5072EB4B28BBF57
:100490003C4615461D46A40098BFA4B208FA04F9CC
:1004A00025EA0909A51C0EFA05FA01FA04F54AEA3B
:1004B000050444EA0904082E2CBF234622460136CF
:1004C0000437102EBFB2DCD102604360BDE8F08774
:1004D000024A136843F080731360704700100240B3
:1004E000062827D8DFE800F004090E13181D2200A3
:1004F000114A13689B01FCD570470F4A1368180115
:10050000FCD570470C4A13689900FCD570470A4A1D
:1005100013689B03FCD57047074A13689807FCD5FE
:100520007047064A13689907FCD57047044A136858
:100530009B07FCD5704700BF00100240201002400E
:100540002410024006281FD8DFE800F004060B1034
:1005500015171900FFF7BCBF0C4A136843F08063FE
:1005600011E00A4A136843F080530CE0074A13680D
:1005700043F4803307E0054A02E0054A00E0054AFB
:10058000136843F001031360704700BF001002407E
:100590002010024024100240034A136823F0030392
:1005A00018431060704700BF04100240034A1368EC
:1005B00023F4701343EA8040106070470410024037
:1005C000034A136823F4803343EA00401060704705
:1005D00004100240034A136823F4404343EA803086
:1005E0001060704704100240034A136823F46053FC
:1005F00043EAC0201060704704100240034A1368A9
:1006000023F4E06343EA00201060704704100240C6
:10061000034A136823F0F00343EA001010607047A8
:100620000410024008B50420FFF78CFF0420FFF7F8
:1006300057FF0020FFF7B0FF0020FFF7E9FF03207E
:10064000FFF7C8FF0420FFF7D9FF0020FFF7CCFF1A
:100650000F4A0120136843F48003136000F03AF856
:100660000A20FFF7A3FF0020FFF7AAFFFFF730FFE4
:100670000020FFF735FF0220FFF78EFF054B064AEB
:1006800006491360064A1160064A136008BD00BFA0
:1006900004100240006CDC021400002000366E01E1
:1006A000180000201C00002001617047090401614E
:1006B00070470368194301607047430903F18043A1
:1006C00003F50433196800F01F00012282400A4339
:1006D0001A607047034A136823F007031843106039
:1006E000704700BF00200240054A136843F08003B2
:1006F0001360044B044A1A6002F188321A60704792
:10070000102002400420024023016745024A13687A
:1007100043F08003136070471020024008B5FFF7D4
:1007200025FEC307FBD408BD2DE9F0411E46036832
:100730000546884617469847069BC0F8D850C360C0
:10074000079BC0F800800361BDF8203047608382BA
:10075000084B8660C366084B8366084B43660023DC
:10076000C0F8C430C0F8C830C0F8CC30C0F8D030C1
:10077000BDE8F08157090008B1090008370A0008F0
:10078000D0F8D8305B6A184710B5D0F8D840A468C4
:10079000A446BDE81040604737B50446002503680D
:1007A0008575C575DB7929462A460095FFF7ECFF6C
:1007B000D4F8D83020465B6829469847E3691BB1D6
:1007C00003B0BDE83040184703B030BD10B5D0F8D5
:1007D000D840E469A446BDE81040604710B5D0F8A1
:1007E000D840246AA446BDE810406047D0F8D8300D
:1007F0001B691847D0F8D8309B69184710B50446D4
:1008000000210122FFF7F2FF002384F82C3010BDF5
:1008100038B50368828FC58EDB79AD1A9D42A8BFBB
:100820001D46836BADB21A4400212B460446FFF7E8
:10083000D5FFA84205D02046FFF7E0FF4FF0FF307C
:1008400038BDA38F0344A38738BD38B50368044679
:10085000DD79838F00219D42826B0FD22B46FFF7FB
:10086000B5FF0223226884F82C30D379A16B0B44A6
:10087000A363D279A38F9B1AA38738BDFFF7A6FF86
:10088000032384F82C300023A387A36338BD2DE90C
:10089000F74F04460E4600F1440500F1640800F1EC
:1008A000380900F13C0B00F1400A2F6857B9204687
:1008B000314604F1380204F13C0303B0BDE8F04FC7
:1008C00000F028BB697933782A7919408A4208D127
:1008D000CDF800A0204631464A465B46B84701287D
:1008E00003D908354545E0D1E1E703B0BDE8F08F15
:1008F00010B50369044683638B79CA7943EA0223FE
:100900008387FFF7C4FF70B1A18F204619B1BDE8FE
:100910001040FFF79ABF0B460A46FFF757FF042324
:1009200084F82C3010BD2046BDE81040FFF766BFAC
:1009300070B5002600EBC6056C6C2CB10136042E98
:10094000F8D14FF0FF3070BD85F8481085F8492088
:100950006B64204670BD70B500F13006002505645B
:100960002946324608230446FFF738FF082804D0FA
:100970002046BDE87040FFF741BFE38E1BB194F9FC
:100980003020002A05DA20463146BDE87040FFF7E6
:10099000AFBFA28A9A42EBD32269A587A2632268DD
:1009A000D2799A4234BF0523062384F82C3070BDD7
:1009B00090F82C3010B5062B044610D0072B24D00D
:1009C000052B33D1FFF724FF002833DBA28FE38E02
:1009D0009B1A2268D27993422CDC062310E0FFF7A1
:1009E00017FF002826DB204604F13001FFF74FFFF8
:1009F00048B100210B4620460A46FFF7E7FE0423D4
:100A000084F82C3010BD204610E000210B460A4629
:100A1000FFF7E4FE002384F82C30236C1BB1204642
:100A200004F1300198470023236410BDBDE8104055
:100A3000FFF7E4BE10BD90F82C3010B5032B044630
:100A400007D0042B07D0022B1CD1BDE81040FFF7C4
:100A5000FCBE072313E0036C13B100F1300198478B
:100A600094F8303053B994F83130052B06D1D4F8CE
:100A7000D830618E5B682046C9B29847002384F85D
:100A80002C3010BDBDE81040FFF7B8BE1988012911
:100A900084BF012119801368C27D01201A7070473C
:100AA00030B5C57D0D246C4340680D3C20448D88D5
:100AB0000479A5420CD201241C808B88D0F809004F
:100AC0001B011B58126803B11B781370012030BD45
:100AD000002030BD19880120022984BF022119801D
:100AE000116800230B701268537070471988012039
:100AF000022984BF02211980116800230B7012683B
:100B00005370704738B514461A882568022A84BF86
:100B100002221A808988C9B2FFF76CFE003018BF24
:100B200001202870236800225A70012038BD08B5C2
:100B300089880122C9B2FFF759FE012008BD08B516
:100B400089880022C9B2FFF751FE012008BD10B507
:100B50000B786BB94C887F2C0AD8D0F8D8308475C4
:100B600093F8302032B149885B68C9B2984701E0F8
:100B7000002010BD012010BDF8B54B88C27D044691
:100B80009A420E4618D0C375D0F8D830DB68984723
:100B9000D4F8C43083B100236364E3646365E36520
:100BA00004F1C00504F1D00755F8043F13B1204605
:100BB00071889847BD42F7D10120F8BD70B51E4637
:100BC000C37D0D225A4343680D3A1A448C88137929
:100BD0000D46A34216D9D2F8091022018C186B8851
:100BE00024799C420ED98A580AB1137000E04BB99F
:100BF000D0F8D43013B1A9886A889847002333808D
:100C0000012070BD002070BD2DE9F04F98464B8843
:100C100089B0DFB21B0A022B0546164611D0032B02
:100C200000F0E380012B40F020810268B8F800104A
:100C30003260026812788A4228BF0A46A8F800206B
:100C400011E10369B8F80040136000930D235F437E
:100C5000D0F80490009819F8075009EB0703A54253
:100C600028BF254619462A46019300F0A3FC009BA5
:100C7000641B19F807705E19A4B200230393019B4B
:100C80001A79BDF80C309A4240F2AA801B010593F4
:100C9000019B059AD3F809301344D3F808A0BAF1A0
:100CA000000F13D09AF800903046A14528BFA14606
:100CB00051464A4600F07EFC9AF80030C9EB040425
:100CC0004D441F444E44A4B2ADB2BFB200230293C0
:100CD000019B059AD3F80930BDF808A013441A798E
:100CE00052457AD9152202FB0AFADB68304613F81E
:100CF0000A9003EB0A0BA14528BFA14659464A4674
:100D0000049300F057FC049BDBF80D1013F80A3035
:100D1000C9EB04044D441F444E44A4B2ADB2BFB26B
:100D2000A1B1DBF811903046A145A8BFA1461FFA3A
:100D300089F94A4600F03EFCDBF81130C9EB0404A7
:100D40004D441F444E44A4B2ADB2BFB2002304933D
:100D5000BDF810A09BF8043053453BD9DBF809C01F
:100D6000CAEB0A1A1CF80A900CEB0A03A14528BF2B
:100D7000A146194630464A46CDF81CC0069300F0FD
:100D800019FCDDF81CC0069B1CF80A20D3F80710DC
:100D9000C9EB04044D4417444E44A4B2ADB2BFB2F3
:100DA000A9B1D3F80B903046A145A8BFA1461FFAC0
:100DB00089F94A4600F0FEFB069BC9EB0404D3F810
:100DC0000B304D441F444E44A4B2ADB2BFB2049B9D
:100DD0000133BCE7029B013379E7039B01334DE705
:100DE000009B5F80A8F800503DE0046967B90923C3
:100DF000A3700423E3702370B8F80030042B28BFDD
:100E00000423A8F800302BE08368013F6BB3C2686D
:100E100097422ADA40F209428988914225D153F853
:100E2000270000F03DFC01304000C0B22070B8F84F
:100E300000304FEA8709984228BF18460022A8F8D8
:100E40000000B8F800305B08013B9A4208DAAB6852
:100E500053F80930995C04EB420359800132F0E702
:100E6000032363703460012000E0002009B0BDE876
:100E7000F08F10B5002200F1C00454F8043F2BB1EC
:100E80000132042AF9D14FF0FF3010BD00EB82008F
:100E9000C0F8C410184610BD30B54C78092C07D8DE
:100EA000044D55F824401CB1A446BDE830406047CD
:100EB000002030BDA017000830B54C780B2C07D8A7
:100EC000044D55F824401CB1A446BDE830406047AD
:100ED000002030BDC817000810B54C78012C03D095
:100EE0000AD3032C04D00CE04C8854B9064C04E01F
:100EF0004C8834B9054C00E0054CA446BDE81040D0
:100F00006047002010BD00BF3F0B00082F0B0008FA
:100F1000050B000810B50C7814F0600F12D104F026
:100F20001F04012C0AD005D3022C0BD1BDE81040C0
:100F3000FFF7D2BFBDE81040FFF7AEBFBDE81040DD
:100F4000FFF7BABF002010BD024B41F080011960CD
:100F5000704700BF4C5C004010B50E4A0E4940F689
:100F60003F731468234043F4004343F0800313604D
:100F700043F60F731468234043F4004343F08003A7
:100F800042F8043B8A42EAD10368DB7920335B00F4
:100F9000038310BD045C0040205C004030B5C9B93B
:100FA000354B10241B68012023F4E04323F0400359
:100FB0009BB2002A0CBF20251025054218BF4340D4
:100FC0004000013C80B2F4D143F400432A4843F08E
:100FD000800303600B0624D501F07F01890001F135
:100FE000804101F5B8410B68102423F4E04323F05D
:100FF00040039BB20120002A0CBF2025102505428A
:1010000018BF43404000013C80B2F4D143F4004398
:1010100043F080030B606ABB48F6CF730A68134045
:1010200027E0890042B94CF68F7001F1804303F547
:10103000B8431C682040186001F1804101F5B841B7
:101040000B68102423F4804323F070039BB201202B
:10105000002A14BF4FF480554FF44055054218BF85
:1010600043404000013C80B2F2D143F4004343F0DE
:1010700080030B6030BD00BF005C00400B060BD549
:1010800001F07F01890001F1804101F5B841086854
:1010900000F03000102809E0890001F1804101F5DD
:1010A000B841086800F44050B0F5805F14BF0020DC
:1010B0000120704701F07F01880000F1804000F5B9
:1010C000B840F0B5046804F03004302C3CD01F4E1A
:1010D000C9003468A4B20C44640004F1804404F5EF
:1010E000C04425685C1CADB26D00641005EB84043F
:1010F00005F1804704F1804407F5C04704F5C0447A
:10110000A74204D032F8025B27F8045BF8E73268A4
:10111000102492B211440E4A490053500268012132
:1011200022F4E04222F0400292B211F0300F18BFD8
:101130004A404900013C89B2F7D142F4004242F0F2
:10114000800202601846F0BD0020F0BD505C0040F7
:10115000046000402DE9F0418C0004F1804404F566
:10116000B844206800F44050B0F5405F56D02E4897
:10117000CE0005682D4FADB235446D007D59C5F3E5
:1011800009059D42054608DA036800F56F709BB2B9
:1011900033445B00C358C3F309032868244D80B26D
:1011A0003044400028585E0880B2400000F1804082
:1011B00000F5C04007469646354603F0010C35B1B0
:1011C00037F8048B013D2EF8028BADB2F7E7BCF186
:1011D000000F03D010F8260002F8160040F60F7238
:1011E0002068024042F080022260124A525CC2B97A
:1011F0002268102022F4804222F0700292B2012173
:1012000011F4405F18BF4A404900013889B2F7D154
:1012100042F4004242F08002226002E00020BDE879
:10122000F0811846BDE8F081505C00400C60004041
:101230000860004024090020F8B5324B05461968C3
:101240001C468EB216F4806F08D04FF6FF321A603B
:1012500040230383BDE8F840FFF79EBA080432D567
:1012600001F00F0116F010034FEA810209D002F1DC
:10127000804303F5B8431B68C3F3C0230133DBB2DB
:101280000CE040F60F7002F1804707F5B847D7F839
:1012900000E00EEA000040F40040386001EB41003D
:1012A000034405EB83035B6E13B1284698470AE0BD
:1012B00002F1804340F60F7203F5B84319680A4003
:1012C00042F080021A60310505D54FF2FF732360AA
:1012D0002B6A03B19847F20405D54EF6FF732360DD
:1012E0006B6A03B19847B30505D54FF6FF532360EA
:1012F000AB6A03B19847AA6A034B02B101221A6094
:10130000F8BD00BF445C004000900B4208B508489F
:101310004FF40001FFF7CDF9064A07490023136097
:101320000B6041F80C3C4FF41C431360034808BDAC
:101330001C100240405C0040505C00402C08002023
:101340002DE9F7430F466C4657490546086849683A
:1013500027F07F0803C407F07F018C0004F180446C
:1013600004F5B84420680A9E20F4E04020F07F0095
:10137000084380B2206048F68F10276808F0FF0C01
:10138000384002AF07EB420232F8082CDFF81CE1CC
:1013900002432260CF00B8F1000F1AD1C9B1DEF8C4
:1013A0000020288B92B23A44DFF804C152003E2B51
:1013B0004CF802001A4644D913F01F0F18BFA3F1CE
:1013C00020026FEA82526FEA5242DEF800E092B2E7
:1013D0003EE0DEF80020288B92B23A44520002F13F
:1013E000804202F5C04210601EB10C2202FB015285
:1013F000566648F6CF72D4F800804FF0100908EA1C
:101400000202226022684FF0010822F4E04222F03A
:10141000400292B218F0200F18BF88EA02024FEA89
:101420004808B9F101091FFA88F8F3D142F40042E3
:1014300042F08002184422602883BCF1000F30D1B2
:10144000ADE713F0010F18BF5A1CDEF800E092025E
:101450001FFA8EFE7744DFF85CE07F004EF807202D
:101460001EB10C2202FB01518E664CF68F72216870
:1014700010260A4022602268012122F4804222F0D4
:10148000700292B211F4405F18BF4A404900013E19
:1014900089B2F7D142F4004242F080020344226054
:1014A0002B8303B0BDE8F083F8170008505C0040C0
:1014B000086000400C6000400B0626D4134B10203F
:1014C0005A54890001F1804101F5B8410B6823F4B9
:1014D000804323F070039BB24AB1012212F4005FF3
:1014E00018BF53405200013892B2F7D108E00122F0
:1014F00012F4405F18BF53405200013892B2F7D146
:1015000043F4004343F080030B607047240900203C
:10151000FEE77047184C19491948002253188342B6
:1015200003D2135953500432F8E7164A002193426C
:1015300002D219600433FAE7134A144C1368144DAD
:1015400043F400731360AC4203D254F8043B984751
:10155000F9E7104C104DAC4203D254F8043B9847C5
:10156000F9E7FEF79DFE0D4C0D4DAC4203D254F849
:10157000043B9847F9E700BF34180008000000203A
:10158000200000202C09002014ED00E03418000891
:1015900034180008341800083418000834180008FB
:1015A00034180008014A024B1A60FEE70400FA05ED
:1015B0000CED00E0844641EA000313F0030349D137
:1015C000403A23D30B6803604B6843608B688360A9
:1015D000CB68C3600B6903614B6943618B698361AD
:1015E000CB69C3610B6A03624B6A43628B6A836295
:1015F000CB6AC3620B6B03634B6B43638B6B83637D
:10160000CB6BC36340304031403ADBD230320BD336
:101610000B6803604B6843608B688360CB68C36072
:1016200010301031103AF3D20C3205D351F8043B8C
:1016300040F8043B043AF9D2043208D0D2071CBF68
:1016400011F8013B00F8013B01D30B880380604691
:10165000704700BF082A13D38B07B1D010F00303E3
:10166000AED0C3F10403D21ADB071CBF11F8013B53
:1016700000F8013BA4D331F8023B20F8023B9FE77E
:10168000043AD9D3013A11F8013B00F8013BF9D2F1
:101690000B7803704B7843708B788370604670478B
:1016A00020F0030110F00300C0F1000051F8043BEA
:1016B00000F1040C4FEACC0C6FF000021CBF22FAC0
:1016C0000CF213434FF0010C4CEA0C2C4CEA0C4C7E
:1016D000A3EB0C0222EA030212EACC1204BF51F877
:1016E000043B0430F4D0C2F1000102EA0102B2FA74
:1016F00082F2C2F11F0200EBD20070471201000219
:101700000000004034127856000201020301090271
:101710000000010100C0321C17000800000000009A
:1017200001000000000000002C1700080904000060
:1017300000FE01020400000000411700080900003B
:1017400000092101FF0000041A0143616262616720
:1017500065732061726520676F6F6420666F722009
:10176000796F75006669736800736F757000404922
:101770006E7465726E616C20466C61736820202007
:101780002F307830383030303030302F382A303009
:10179000314B612C35362A3030314B670000000068
:1017A000D50A000800000000000000000000000052
:1017B000000000004F0B0008090C000800000000AA
:1017C0008D0A0008790B0008ED0A000800000000EF
:1017D0000000000000000000000000000000000009
:1017E00000000000000000000000000000000000F9
:1017F000A10A0008BD0B000800020004000000065A
:101800000D130008490F000841130008590F000884
:101810009D0F0008B91400087D100008B5100008DD
:1018200055110008391200080000000000000000F7
:0418300000000000B4
:10183400020000004A17000864170008691700082E
:101844006E17000800127A0000127A0000127A0063
:0400000508001515C5
:00000001FF
